:100000001EC036C035C034C033C032C031C030C06D
:100010002FC02EC065456A466E47734878497D609B
:10002000826187628C63906495659A669F67A46815
:10003000A969AE80B381B782BC83C184FF2111243A
:100040001FBECFE9CDBF10E0A0E6B0E0E4E3F3E0EF
:1000500002C005900D92A037B107D9F710E0A0E7D4
:10006000B0E001C01D92A137B107E1F735D060C102
:10007000C7CF2AE134E003C0F9013197F1F70197C6
:10008000D8F708958EE591E00197F1F70895369A33
:100090003699FECF85B10895EF92FF920F931F938B
:1000A000CF93DF93F82EEB018B01000F111F000F90
:1000B000111F95E2E92E07C0E9BCCE01DADF19BCB9
:1000C000C801D7DFFA94F110F7CFDF91CF911F91DC
:1000D0000F91FF90EF90089582E087BBA29A81E68E
:1000E00087B986EC86B9479A85B7877E85BF8091A8
:1000F0007200882329F0109271001092700013C0D2
:100100008091710080937000809170008F5F809368
:100110007000809170008F3010F01092700080910C
:1001200070008093710010927200E0917000F0E016
:10013000E05AFF4F80818A3010F481E201C083E2EF
:100140008FBD81E083BFE0917000F0E0E05AFF4F87
:10015000808189BDC0E0DFEF14E602E48091700089
:10016000853040F485B7806285BF889585B78F7DDF
:1001700085BFB2C080917000863070F519BC87DFF2
:1001800088EC90E076DF83DF90E001C09E5F292F4E
:1001900030E0F901EC5EFF4FE491E817B8F3F901A4
:1001A000EB5EFF4FF4906EE370E08F2D82958695A5
:1001B000877072DF84EF91E05CDF65E070E081E0E2
:1001C0006BDF8EEE92E055DF6EE370E08F2D8F7166
:1001D00063DF80ED97E07FC080917000873080F40E
:1001E000D9BD81E090E045DF19BC89EF90E041DFA7
:1001F000D9BD81E090E03DDF19BC8DEE92E06BC08F
:10020000809170008A30B8F4D9BDE0917000F0E0C0
:10021000E05AFF4F8081823310F434DF03C081E065
:1002200090E027DF19BCE0917000F0E0E05AFF4F4A
:10023000808190E050C0809170008A30B9F4F12C38
:10024000D9BD81E090E015DF19BC80E28F1518F46C
:10025000802F8F1901C08F2D90E04B96880F991F2A
:1002600008DFF39482E4F812EBCF36C0809170007F
:100270008B3099F4F12CD9BD05DF19BC81E38F15C2
:1002800018F4812F8F1901C08F2D90E00996F1DEAF
:10029000F39484E6F812EFCF1FC0809170008F3086
:1002A000D8F424E0F22EE0917000F0E0E35AFF4F22
:1002B000808189BD85E090E0DCDEE0917000F0E0B7
:1002C000E05AFF4F808189BD81E490E0D2DEFA944C
:1002D00051F780ED92E0CDDE349B40CFD8DE90E048
:1002E00020917000211103C02EE630E002C023E708
:1002F00030E082179307CCF4CF5FC330B8F0809121
:100300007000882319F0109270000CC019BC85B7DA
:10031000877E806185BF85B7806285BF889585B7F8
:100320008F7D85BF88EE93E0A4DEC0E0369A16CFBD
:04033000F894FFCF6F
:10033400040E256EFF25FF52290FFFFF040E250032
:00000001FF
